:100000000C9483040C94C7040C94C7040C94C70488
:100010000C94C7040C94C7040C94C7040C94C70434
:100020000C94C7040C94C7040C94DB190C94AD1AFF
:100030000C9414280C94C7040C94C7040C94C704A3
:100040000C94C7040C94F0050C94C7040C94C704DA
:100050000C94C7040C947C280C94C7040C94C7041B
:100060000C94C7040C94C7040C94C7040C94C704E4
:100070000C94C7040C94C7040C94C7040C94C704D4
:100080000C94940F0C94C7040C94C7040C94C704EC
:100090000C94C7040C94C7040C94C7040C94C704B4
:1000A0000C94C7040C94C7040C94C7047A068D06FC
:1000B000A206B506BD06D306E906F206FC0607074A
:1000C00010071907210729073C073C073C073C0795
:1000D0003C073C07370758063C076006690672066E
:1000E0001A1B3C1B2A1C3C1B2A1C811BA41B2A1C00
:1000F000F91B0C1CFB1EFB1E2A1F2A1F691F891FD0
:10010000DF20DF20941FDF2044204420AB20B420D8
:10011000DF20D92051205120512051205120512041
:100120005120512051205120512051205120512047
:100130005120512061206F2076207D208720B02D16
:10014000A62DB92D112E182E182E112E182E182E60
:10015000DE2D182EE82DF22D182E182E182E182E02
:10016000112E182E182E112E182ECB2D182E182EBB
:10017000FD2DFD2DFD2DFD2DFD2DFD2DFD2DFD2D2F
:10018000FD2D132E182E132E182E182E182E182E65
:10019000182E182E182E182E182E182E182E132E34
:1001A000182E182E112E902DFB2DFB2DFB2DFB2D27
:1001B000FB2DFB2DFB2DFB2DFB2D132E0763423654
:1001C000B79BD8A71A39685618AEBAAB558C1D3CE8
:1001D000B7CC5763BD6DEDFD753EF6177231BF00AC
:1001E0000000803F08000000BE922449123EABAAE6
:1001F000AA2ABECDCCCC4C3E00000080BEABAAAA41
:10020000AA3E00000000BF000000803F0000000088
:1002100000084178D3BB4387D1133D190E3CC3BDC1
:100220004282AD2B3E68EC8276BED98FE1A93E4C6E
:1002300080EFFFBE01C4FF7F3F0000000000000010
:10024000000000000000000000010204060A0F1771
:10025000202C3A4A5D71879DB3C7DAE9F5FCFFFCB3
:10026000F5E9DAC7B39D87715D4A3A2C20170F0A6A
:10027000060402010000000000000000000000224F
:1002800029001E001F00200021002200230024005E
:100290002500260027002D002E002A002A002B0012
:1002A00014001A000800150017001C0018000C00AC
:1002B000120013002F00300031004C003900040000
:1002C0001600070009000A000B000D000E000F00C9
:1002D00033003400280028004B00E1001D001B0003
:1002E0000600190005001100100036003700380024
:1002F000E500E50052004E00E000E3000530E200BA
:1003000003302C002C000430C000E6006500E4003F
:10031000500051004F0029001E001F002000210046
:100320002200230024002500260027002D002E0097
:100330002A002A002B0014001A00090013000A00EA
:100340000D000F0018001C0033002F00300031009A
:100350004C002A00040015001600170007000B00CF
:10036000110008000C0012003400280028004B0087
:10037000E1001D001B000600190005000E00100022
:10038000360037003800E500E50052004E00E0007E
:10039000E3000530E20003302C002C000430C000E4
:1003A000E6006500E400500051004F0029001E00E7
:1003B0001F00200021002200230024002500260029
:1003C00027002F0030002A002A002B0034003600BE
:1003D000370013001C0009000A00060015000F007A
:1003E00038002E0031004C003900040012000800D3
:1003F00018000C0007000B001700110016002D005C
:10040000280028004B00E100330014000D000E000E
:100410001B00050010001A0019001D00E500E50092
:1004200052004E00E000E3000530E20003302C00F3
:100430002C000430C000E6006500E40050005100CC
:100440004F004600153017301830193000000000FA
:1004500053005400550000000000470048004800C9
:1004600001003A003B003C003D00000000005F003E
:1004700060006100560001000100010049003900E0
:100480003E003F0040004100000000005C005D00B5
:100490005E0057000100010001004A000100420017
:1004A0004300440045000000000059005A005B0072
:1004B00058000100010001004D0001000100010091
:1004C00001000100620062000100E60063005800C4
:1004D000010001000100010001003A003B003C0066
:1004E0003D003E003F004000410042004300440008
:1004F000450001000100010021022F022F00260209
:10050000220220022702300030021F0201000100F7
:100510000100490001002302250257005600330064
:1005200033022D02340034023500010001000100C5
:100530004A000100310224021E0235023800310057
:100540002E003602370238020100010001004D0082
:100550000100010001000100010001000100010093
:100560000100010001000100010001000100530031
:100570003A003B003C003D003E003F00400041008F
:1005800042004300440045000100010047006800AC
:1005900069006A006B006C006D006E006F007000F7
:1005A0007100720073000100480039000100010071
:1005B0000100010001000100010001000100010033
:1005C00001000100010046000100010001000100DE
:1005D0000100010001000100010001000100010013
:1005E0000100A900A80001000100010001000100B4
:1005F000AE00AE0001000100010001000100AC00EE
:10060000AA00AB000100FD00FE00FF00000000009A
:1006100000000000000000000000000000000000DA
:1006200000000000000000000000000000000000CA
:1006300000000000000000000000000000000000BA
:100640000000F800F700F600F500000000000000D0
:10065000000000000000000000000000F9000100A0
:10066000000000000000000000000000000000008A
:100670000000000001000100F000FA00010001008C
:10068000010001000100F400F4000100010001007C
:1006900001000100F200F100F30001000730083012
:1006A00009300A300B300C300D3001000100010020
:1006B00025502250010001000100003001300230BD
:1006C0000100010001000100010001000100010022
:1006D0000100010001000100010001000100010012
:1006E0000100010001000100010001000100010002
:1006F0000100010001000100010001001430005060
:100700000100063001000100010001000100265037
:1007100001000100010001000100010001000100D1
:10072000010001000100010001000100275001004B
:1007300028035400680065002000410074006F0029
:100740006D006900630020004B00650079006200C5
:100750006F0061007200640000002C034F00720003
:10076000740068006F006C0069006E006500610035
:10077000720020004B006500790062006F0061008C
:1007800072006400730000000403090409026D0094
:10079000040100A0FA09040000010301010009217D
:1007A00011010001223F000705810308000A090426
:1007B00001000103010200092111010001224D0085
:1007C0000705820308000A09040200010300000073
:1007D0000921110100012236000705830308000AE0
:1007E0000904030001030000000921110100012296
:1007F00039000705840310000112011001000000F8
:1008000008EDFE190401000102000105010906A11D
:1008100001050719E029E7150025019508750181F3
:1008200002050819012905950575019102950175C3
:1008300003910105071900297715002501957875A1
:10084000018102C005010980A1018502160100266F
:10085000B7001A01002AB700751095018100C00584
:100860000C0901A1018503160100269C021A010052
:100870002A9C02751095018100C005010902A101A1
:100880000901A10005091901290515002501950592
:100890007501810295017503810105010930093156
:1008A0001581257F95027508810609381581257FF8
:1008B000950175088106050C0A38021581257F957A
:1008C0000175088106C0C005010906A101050719C7
:1008D000E029E7150025019508750181029501754C
:1008E00008810105081901290595057501910295F1
:1008F00001750391010507190029FF150025FF95D2
:100900000675088100C011241FBECFEFDAE0DEBFFC
:10091000CDBF04B603FE24C080917B0590917C0579
:10092000A0917D05B0917E058730904BA740B04BDC
:10093000B9F410927B0510927C0510927D051092FF
:100940007E0514BE84B7877F84BF88E10FB6F89414
:1009500080936000109260000FBEE0E0F8E309951C
:1009600014E0A0E0B1E0EEE0F7E602C005900D92E1
:10097000A431B107D9F715E0A4E1B4E001C01D929C
:10098000AB37B107E1F70E9421170C9485330C9423
:100990000000089581E008950C94C9040C94CA04E1
:1009A0000C9441070E944F2F811105C0109216042C
:1009B000109215040DC080E290E00090170402C070
:1009C000880F991F0A94E2F79093160480931504F8
:1009D0001092140480916F00826080936F000895DC
:1009E0000E944F2F811105C0109216041092150419
:1009F0000DC081E290E00090170402C0880F991F9B
:100A00000A94E2F7909316048093150482E0809391
:100A1000140480916F00826080936F0008950E949B
:100A20004F2F811102C081E001C082E08093140445
:100A3000089590916F0081E0911101C080E00895C8
:100A40000E944F2F23E030E0281B3109220F209312
:100A500018040895282F2F9880918000211108C034
:100A6000877F8093800010928D0010928C001BC0B5
:100A7000886080938000233018F08FEF9FEF0FC0C5
:100A800083E090E0821B9109880F991F2FEF3FEFC1
:100A9000A90102C0569547958A95E2F7CA0190933D
:100AA0008D0080938C000C9420050E941905811103
:100AB00018C00E944F2F811105C010921604109289
:100AC00015040DC081E290E00090170402C0880F69
:100AD000991F0A94E2F790931604809315041092DC
:100AE000140490916F0082E0892780936F000E9428
:100AF0001905811104C00E944F2F0C942A050895F6
:100B0000CF93C82F0E94190540911704882329F01C
:100B100090916F009D7F90936F00C093170488237E
:100B2000D1F0209115043091160402C03695279516
:100B30004A95E2F72F733327C90102C0880F991F26
:100B4000CA95E2F7909316048093150480916F0084
:100B5000826080936F00CF91089590911704292FA0
:100B600030E0281B31092B30310510F080E002C045
:100B7000981B892F0C94800590911704282F30E042
:100B8000290F311D2B30310514F08AE001C0890F87
:100B90000C9480050E94200584E080931704109235
:100BA00014040895279A2F988FEF9FEF9093870052
:100BB000809386008AE08093800089E180938100A1
:100BC0000E94B82E0C94CA0585B7806885BF85B78A
:100BD000806885BF0E94D2056E9A769A0C94B607FB
:100BE0001F920F920FB60F9211242F933F938F9362
:100BF0009F93EF93FF93E0911504F0911604CF01BA
:100C0000019690931604809315040090170402C077
:100C1000F695E7950A94E2F7EF7380911404823019
:100C200019F4E03251F404C0813039F4EF3329F47F
:100C300080916F008D7F80936F00F0E0E25CFD4F4C
:100C4000E49121E031E0E29FC001E39F900D112487
:100C50000090180402C0969587950A94E2F7909345
:100C60008D0080938C00FF91EF919F918F913F9128
:100C70002F910F900FBE0F901F901895CF93DF9379
:100C8000EC010E94702ABE0180E090E0DF91CF91DC
:100C90000C940A250F931F93462F50E04A315105BB
:100CA00008F0EAC0DC01FA01EA5AFF4F0C9449331C
:100CB00012968C91882309F4DFC00E945505DCC090
:100CC00012968C91882309F4D7C081E00E94AD056B
:100CD000D3C012968C91882309F4CEC081E00E9483
:100CE000BC05CAC012968C91882309F4C5C00E9425
:100CF000CA05C2C012968C91882309F4BDC081E058
:100D000090E00E943E060AE017ED23E23CE340E05B
:100D100064E070E080E792E012C012968C91882324
:100D200009F4AAC082E090E00E943E060AE017EDB6
:100D300023E23CE340E066E070E080E092E00E9465
:100D400012139AC012968C91882309F495C084E0FE
:100D500090E00E943E060AE017ED23E23CE340E00B
:100D600068E070E080E392E0EACF12968C918823ED
:100D700011F083E007C083E013C012968C918823A2
:100D800071F084E00E94872582E00E9480050E9425
:100D9000F00447E063E084E00E94840D6DC084E0CD
:100DA0000E94A825F6CF12968C91882349F083E003
:100DB0000E9480050E94D20485E00E9487255CC0C5
:100DC00081E00E9480050E940F0585E00E94A82511
:100DD00053C012968C91882309F44EC086E00E947D
:100DE000CD254AC012968C91882309F445C060E055
:100DF00070E080E09EE308C012968C918823E1F1B8
:100E000060E070E080E89EE30E94BC1335C012965B
:100E10008C91882389F160E070E080E09FE3F4CF5B
:100E200012968C91882341F160E070E080E49FE3AA
:100E3000EBCF12968C918823F9F08AE00E94CE13B2
:100E40001BC012968C918823B9F08AE00E94C813C7
:100E500013C012968C91882379F060E070E080E0F6
:100E60009FE30E94BC1384E60E94C51305C012963E
:100E70008C9181110E940F2F80E090E01F910F91C3
:100E800008950F931F93CF93C82F8FE39CE9019789
:100E9000F1F700C000000E94A51381114BC0909192
:100EA0001904C1FF0BC091FD14C000E010E09801CF
:100EB00040E062E070E080E591E03AC091FF09C057
:100EC00000E010E0980140E062E070E080E491E032
:100ED0002FC0C0FF0BC090FD14C000E010E09801CF
:100EE00040E062E070E080E391E022C090FF09C042
:100EF00000E010E0980140E062E070E080E291E004
:100F000017C0C2FF0BC092FD15C000E010E09801B1
:100F100040E062E070E080E191E00AC092FF0AC028
:100F200000E010E0980140E062E070E080E091E0D5
:100F30000E941213C0931904CF911F910F9108952D
:100F40000F931F938FE39CE90197F1F700C0000016
:100F50000AE017ED23E23CE340E06FE070E088ED4B
:100F600092E00E9412131F910F91089580E00E9459
:100F7000DF130C94A0070F931F930AE017ED23E2F1
:100F80003CE340E069E070E080E992E00E941213E7
:100F90002FEF87EA91E6215080409040E1F700C0B2
:100FA00000001F910F910C94C70E0F931F930AE03E
:100FB00017ED23E23CE340E065E070E088ED91E06E
:100FC0000E9412131F910F9108950F931F930AE02F
:100FD00017ED23E23CE340E067E070E080EA91E057
:100FE0000E9412131F910F9108950F931F930AE00F
:100FF00017ED23E23CE340E068E070E080E691E03A
:101000000E9412131F910F91089581E008950C948E
:10101000050808950C94E40580916A04882309F476
:1010200048C08091260490912704009779F40E948B
:10103000462890932704809326048091280490E00A
:10104000009771F48091290490E00AC00E94522810
:1010500020915003309151032817390740F329C0DC
:101060000197880F991F880F991FFC01E65DFB4FC0
:1010700060817181828193810E94FA0EE09128043F
:1010800084E0E89FF0011124E65DFB4F60817181EF
:10109000828193814FE050E00E94B2128091280437
:1010A00090E001966091290470E00E9435338093AE
:1010B00028040C94CC0410926C040C94C70E81E0AC
:1010C00080936C040C94E5078F929F92AF92BF922D
:1010D000EF92FF920F931F93CF93DF93CDB7DEB7BD
:1010E000A3970FB6F894DEBF0FBECDBF7C01FC0105
:1010F00000811181C8010E944326B8010E94660A3E
:101100008C01B7010E940708882309F4CCC1003282
:10111000F0E51F0741F4F7018281882309F458C0E4
:101120000E94AC13C0C10132F0E51F0741F4F70182
:101130008281882309F44CC00E94B513B4C10232E5
:10114000F0E51F0751F4F7018281882309F440C0BC
:101150000E94A8138111F0CFE3CF0332F0E51F07FF
:1011600039F4F7018281882399F10E945F089BC1BD
:101170000432F0E51F0739F4F7018281882341F139
:101180000E945B0890C10532F0E51F0749F4F701A2
:1011900082818823E9F080916C048111F1CFE5CF41
:1011A0000632F0E51F0739F4F7018281882381F0C8
:1011B0000E94E2130AC00732F0E51F0749F4F70165
:1011C0008281882329F00E94ED130E94F5076BC1EC
:1011D00080916C04811105C0F70182818111CFC01B
:1011E00018C1003E110579F4F7018281882309F4C2
:1011F0004DC00E94C70E81E080936B0410926A0478
:101200001092290450C1023E110559F4F701828160
:101210008823E1F10E94C70E10926B0410926A04B9
:1012200042C1033E110591F4F7018281882371F1D7
:101230000E94C70E10926B0481E080936A041092A2
:10124000280410922704109226042DC1023511059E
:1012500059F4F7018281882309F425C18091500354
:10126000909151030A970DC00135110579F4F701EA
:101270008281882309F417C1809150039091510312
:101280000A9690935103809350030DC140915403EB
:1012900083E2EFE6F3E0DE01119601900D928A956C
:1012A000E1F7F701808121E030E02C0F3D1F280F8E
:1012B000311DC9012091520330915303FC01E20F0B
:1012C000F31F6081772767FD7095640F711D882774
:1012D00077FD8095982F0E94573020E030E040E461
:1012E00051E40E94BC2F4B015C01F701218185E094
:1012F00090E0821B9109BC01882777FD8095982F8B
:101300000E9457309B01AC01C501B4010E94542FCB
:101310009B01AC0160E070E080E090E40E94CA3183
:1013200020E030E04CED50E40E9467314B015C015D
:10133000F70182818823D1F04FE050E0C501B4016C
:101340000E94B21280916B048823A1F0809129043D
:1013500024E0829FF0011124E65DFB4F80829182A0
:10136000A282B3828F5F8093290404C0C501B401B7
:101370000E94FA0E0F3F110508F02ECF94C0809105
:10138000250481111FC0043130E5130709F051C055
:101390000E94090881E0809325040E9446289093CA
:1013A00024048093230410921C0410921E041092B3
:1013B0001D041092200410921F0410922204109217
:1013C000210471C080912304909124040E9452282A
:1013D000883C910570F480911C04E82FF0E0EE0F3A
:1013E000FF1FE35EFB4F118300838F5F80931C041C
:1013F0005AC0043880E5180721F00538104501F17E
:101400003AC0F7018281882341F010921A0482E0E9
:101410001EC0043830E5130759F580911A04811174
:1014200006C086E20E949F1D86E20E94671E82E03F
:101430001CC00438F0E51F0741F305381045D9F406
:10144000F7018281882331F010921B0480E20E9410
:10145000B61E29C080911B04811106C087E20E943C
:101460009F1D87E20E94671E80E20E94BD1E1BC076
:101470000538104529F381E080931A0480931B04FA
:10148000C701A3960FB6F894DEBF0FBECDBFDF91A4
:10149000CF911F910F91FF90EF90BF90AF909F90D1
:1014A0008F900C94CE0480E0A3960FB6F894DEBF24
:1014B0000FBECDBFDF91CF911F910F91FF90EF90A5
:1014C000BF90AF909F908F90089508959FE0799F6F
:1014D000F00111249BE4899FE00DF11D1124E60F1A
:1014E000F11DEE0FFF1FE058FD4F85919491089577
:1014F000880F991FFC01E250FF4F85919491089548
:10150000880F991FFC01E258FD4F85919491089531
:101510000F931F93CF93DF93EC01811521E3920783
:10152000A0F5C11580E3D80708F0D7C0C83ED105A3
:10153000D8F4C03ED10508F007C2C83AD10578F406
:10154000C53AD10508F06AC0C130D10509F463C0BD
:1015500008F4F7C1C430D10508F0F6C1F2C1CB3BA5
:10156000D10508F466C0EDC1C11590E2D90708F0B5
:10157000AFC0C11521E0D20708F0E6C1C03FD105D8
:1015800008F4DFC18E0110651FC2C03880E5D8079E
:1015900000F5C03790E5D90708F0A3C0C11520E5D4
:1015A000D20709F4ACC050F4CE01905480319F4072
:1015B00008F0C7C1DF708E01106A06C2C13080E535
:1015C000D80709F4AEC0C43190E5D90708F4AFC01C
:1015D000B8C1C33820E5D20709F48EC050F4C13831
:1015E00090E5D90709F482C008F083C000E011ED4E
:1015F000EBC1C03181E5D80708F4A3C1C11597E557
:10160000D90708F436C1CE0190578115904108F0F2
:1016100098C1DF7093C101E010E0D6C1C53AD10591
:1016200009F494C1C63AD10509F093C102E810E467
:10163000CBC1C83AD10509F48FC1C93AD10509F423
:101640008EC1CA3AD10509F48DC1CB3AD10509F44E
:101650008CC1CC3AD10509F48BC1CD3AD10509F43E
:101660008AC1C03BD10509F489C1CE3AD10509F43C
:1016700088C1CF3AD10509F487C1C13BD10509F42E
:1016800086C1C23BD10509F485C1C33BD10509F42C
:1016900084C1C43BD10509F483C1C53BD10509F41C
:1016A00082C1C63BD10509F481C1C73BD10509F40C
:1016B00080C1C83BD10509F47FC1C93BD10509F4FC
:1016C0007EC1CA3BD10509F47DC100E014E47CC1B0
:1016D000CE019F700E94800A78C1DD278E01106CB8
:1016E00073C1CF70DD278E01146D6EC100E010ED67
:1016F0006BC100E012ED68C100E013ED65C10E940E
:101700004A210E94C70E0E94BB078FEF94E32CE092
:10171000815090402040E1F700C000000E94A128C5
:1017200053C180914D05816080934D054DC10E944C
:10173000582A811102C00E94342A0E94752A90E022
:1017400090937A0580937905C23080E5D80721F41B
:1017500080917905816086C0C43090E5D90721F475
:101760008091790582607EC0C63020E5D20721F4E1
:1017700080917905846076C0C83080E5D80719F477
:101780008091790527C0CA3090E5D90721F480916E
:101790007905806167C0CC3020E5D20721F48091C3
:1017A000790580625FC0CE3080E5D80721F4809152
:1017B0007905806457C0C03190E5D90721F4809144
:1017C000790580684FC0C23120E5D20729F48091A5
:1017D00079058460886046C0C33080E5D80721F46D
:1017E000809179058E7F3EC0C53090E5D90721F400
:1017F000809179058D7F36C0C73020E5D20721F46E
:10180000809179058B7F2EC0C93080E5D80719F407
:101810008091790526C0CB3090E5D90721F48091DD
:1018200079058F7E1FC0CD3020E5D20721F480914D
:1018300079058F7D17C0CF3080E5D80721F48091DE
:1018400079058F7B0FC0C13190E5D90721F48091D4
:1018500079058F7707C0C331D04531F48091790580
:101860008B7F877F80937905809179050E94792A03
:10187000ABC08D2F99278F70992781309105D9F4AE
:101880009E012370332702C0880F991F2A95E2F723
:101890009C688E0144E0000F111F4A95E1F7002774
:1018A0001370802B912B53E0CC0FDD1F5A95E1F77D
:1018B000C076DD272FC08230910531F4DC2FCC2794
:1018C0008E01016F106A80C08330910569F4CE01EA
:1018D0008370992701E010E002C0000F111F8A9564
:1018E000E2F7C8019C680FC084309105B9F4CE01BD
:1018F0008370992701E010E002C0000F111F8A9544
:10190000E2F7C8019A6823E0CC0FDD1F2A95E1F7C2
:10191000C07ED7708C010C2B1D2B56C085309105D5
:1019200031F4DC2FCC278E01046F106A4DC006976E
:1019300009F04AC0CF71DD27DC2FCC278E01106261
:1019400043C000E010E040C08E013EC001E810E45A
:101950003BC003E810E438C002EE14E435C009EEE1
:1019600014E432C00AEE14E42FC005EB14E42CC0DA
:1019700006EB14E429C007EB14E426C00CEC14E4D5
:1019800023C00DEC14E420C003E815E41DC00AE8F0
:1019900015E41AC002E915E417C004E915E414C0FF
:1019A00001E216E411C003E216E40EC004E216E4FC
:1019B0000BC005E216E408C006E216E405C007E223
:1019C00016E402C00AE216E4C801DF91CF911F912C
:1019D0000F9108959FE0799FF00111249BE4899F66
:1019E000E00DF11D1124E60FF11DEE0FFF1FE05871
:1019F000FD4F85919491803E9105E0F4803C9105E6
:101A000058F58133910509F46FC048F48932910586
:101A100009F463C08A32910509F46DC072C089333C
:101A20009105E9F082389105D1F08533910509F4EB
:101A30004DC067C0833E910581F138F4803E910529
:101A4000B9F0823E9105D9F05CC0863E910561F106
:101A5000873E9105A1F155C00E94780A0895209112
:101A6000790520FD02C021FF4CC080EE90E049C006
:101A70008091790580FFF9CF89E390E042C08091A1
:101A8000790582FF0EC08091790584FF03C080E054
:101A900090E037C083EE90E034C08091790582FFFA
:101AA000F2CF82EE90E02DC08091790583FF0BC0CC
:101AB0008091790584FDEBCF87EE90E022C0809184
:101AC000790583FFF5CF86EE90E01BC08091790504
:101AD00085FF07C089E290E014C08091790585FFF9
:101AE000F9CF85E390E00DC08091790586FF07C0AE
:101AF0008AE290E006C08091790586FFF9CF81E304
:101B000090E00E94880A0895CF92DF92EF92FF92B0
:101B10000F931F9301E010E020E030E068017901AD
:101B200004C0CC0CDD1CEE1CFF1C8A95D2F704C04F
:101B3000000F111F221F331F6A95D2F70C291D2990
:101B40002E293F29C0903005D0903105E090320514
:101B5000F0903305C022D122E222F322842FC01656
:101B6000D106E206F30641F41F910F91FF90EF902A
:101B7000DF90CF900C9487251F910F91FF90EF90ED
:101B8000DF90CF900C94A8250C94D004E82FF0E0BF
:101B9000EF55FC4F8081E82FEF70F0E082958F7059
:101BA00021E030E0A90102C0440F551F8A95E2F7F9
:101BB00040A308950F931F93CF93DF9385B7806859
:101BC00085BF85B7806885BFC4E0D0E001E010E044
:101BD000FE01EF55FC4F8081E82FEF70F0E021A16E
:101BE00082958F70A80102C0440F551F8A95E2F7B5
:101BF000CA01822B81A38C2F0E94C60D219740F72A
:101C00008EE090E061E070E0FC01EE56FC4F208138
:101C1000E22FEF70F0E042A122952F70DB0102C0AD
:101C2000AA0FBB1F2A95E2F79D01242B22A301973F
:101C300058F7DF91CF911F910F910C940A08EF9202
:101C4000FF920F931F93CF93DF9307E714E0C4E055
:101C5000EE24E394F12CD5E08C2F0E94C60D8EE08B
:101C600090E040E050E0FC01EE56FC4F6081E62F32
:101C7000EF70F0E020A130E062956F7002C0359502
:101C800027956A95E2F720FD09C09701082E02C04A
:101C9000220F331F0A94E2F7422B532B019718F7B8
:101CA000F801929182918F018417950721F0518359
:101CB0004083D09355038C2F0E94C60DC15060F60F
:101CC0008091550387FD1FC08150809355038F3F3E
:101CD00039F08FE99FE00197F1F700C0000013C0D1
:101CE00080E090E0FC01E958FB4FDC01A359BB4FB9
:101CF00018962D913C911997318720870297863F3E
:101D0000EFEF9E0779F70E940C0881E0DF91CF91F9
:101D10001F910F91FF90EF900895E82FF0E0EE0FE4
:101D2000FF1FE958FB4F80819181089508950F931B
:101D30001F93CF9301E814E0C0E0F80192918291E3
:101D40008F010E94BE27C80FF4E007371F07A9F7CD
:101D50008C2FCF911F910F9108950E94582A8111C5
:101D600002C00E94342A0E94872A809364053E9A0A
:101D7000809171008D7F8093710082E0809390004C
:101D80008AE18093910081E080938304089580919B
:101D90008304811102C00E94AD0E1092D3041092F0
:101DA000D204809171008D7F8093710080919000AA
:101DB0008F73809390001092950410929404109267
:101DC000CC041092CD041092CE041092CF04109245
:101DD000CB041092CA04EAEAF4E0AAE9B4E0119252
:101DE0001192119211921D921D9284E0EA3CF80723
:101DF000B1F70895CF92DF92EF92FF920F931F9366
:101E0000CF93DF9320919404222309F484C06B01C3
:101E10007C0180918304811102C00E94AD0E0AEC06
:101E200014E0C7E0D0E0A7019601F80192918291F9
:101E3000729162918F010E94B82F811131C0FE0111
:101E4000EE0FFF1FEE0FFF1FE655FB4F10821182B2
:101E500012821382DE01AA0FBB1FA656BB4F11963A
:101E60001C921E92C730D105E9F02196448155811C
:101E700066817781408351836283738314821582E4
:101E80001682178212968D919C91139711969C93AE
:101E90008E9313961C921E92129734961296E2CF4E
:101EA000219708F68091D2049091D304019797FD71
:101EB00005C09093D3048093D20404C01092D3043D
:101EC0001092D2048091D2049091D3042091D00436
:101ED0003091D1042817390724F01092D1041092C0
:101EE000D004892BC1F4809171008D7F80937100A3
:101EF000809190008F73809390001092CC04109288
:101F0000CD041092CE041092CF041092CB04109204
:101F1000CA0410929404DF91CF911F910F91FF900A
:101F2000EF90DF90CF9008951F920F920FB60F920F
:101F300011244F925F926F927F928F929F92AF92F5
:101F4000BF92CF92DF92EF92FF922F933F934F93E6
:101F50005F936F937F938F939F93AF93BF93CF9331
:101F6000DF93EF93FF9380919404882309F49BC13E
:101F7000C091D204D091D3041C161D060CF093C15D
:101F8000409084045090850460908604709087048B
:101F900020E030E0A901C301B2010E9463311816AC
:101FA0000CF065C0C130D10509F452C08091D00455
:101FB0009091D104BE010E9435337C019093D104ED
:101FC0008093D0048090960490909704A0909804F9
:101FD000B090990420E030E040E85FE3C501B4012F
:101FE0000E94542F609396047093970480939804F2
:101FF00090939904F701EE0FFF1FEE0FFF1FE655B8
:10200000FB4FA301920160817181828193810E94C3
:10201000BC2F20E030E040E05EE30E9467319B018E
:10202000AC01C501B4010E94633118168CF4C701DC
:102030000196BE010E9435339093D1048093D00461
:10204000109296041092970410929804109299049A
:10205000E091D004F091D104EE0FFF1FEE0FFF1FAF
:10206000E655FB4F6081718182819381D0C0C09021
:10207000CC04D090CD04E090CE04F090CF0420E0CA
:1020800030E0A901C701B6010E94B82F219788232B
:1020900009F4A2C0FE01EE0FFF1FEE0FFF1FE65571
:1020A000FB4F80809180A280B380A5019401C7017D
:1020B000B6010E94B82F87FF31C0A501940160E0EE
:1020C00070E08CED93EC0E94BC2F20E030E040E407
:1020D00051E40E94BC2F20E030E040E05FE30E942A
:1020E00067319B01AC0160E070E080E090E40E9409
:1020F000CA319B01AC01C501B4010E9467319B014B
:10210000AC01C701B6010E94B82F87FF07C0A70125
:10211000960160E070E08CED93E439C0A501940174
:10212000C701B6010E94633118160CF055C0A50115
:10213000940160E070E08CED93E40E94BC2F20E0FD
:1021400030E040E451E40E94BC2F20E030E040E069
:102150005FE30E9467319B01AC0160E070E080E0CA
:1021600090E40E94CA319B01AC01C501B4010E94F8
:1021700067319B01AC01C701B6010E94633118169B
:102180005CF5A701960160E070E08CED93EC0E9495
:10219000BC2F20E030E040E451E40E94BC2F20E05E
:1021A00030E040E05FE30E9467319B01AC0160E0FA
:1021B00070E080E090E40E94CA319B01AC01C7014D
:1021C000B6010E9467316093CC047093CD04809374
:1021D000CE049093CF0413C0FE01EE0FFF1FEE0F4D
:1021E000FF1FE655FB4F80819181A281B3818093CF
:1021F000CC049093CD04A093CE04B093CF0460910F
:10220000CC047091CD048091CE049091CF042091A4
:102210008104309182042F3F4FEF340731F02F5F5C
:102220003F4F30938204209381040E94F8136B0186
:102230007C0120E034E244EF51E40E94B82F87FF94
:1022400008C086EFC82E88E2D82E84EFE82E81E4FD
:10225000F82E20E030E040E051E4C701B6010E94D2
:1022600067319B01AC0160E074E284E79BE40E946B
:10227000BC2F6B017C010E94293070939700609302
:102280009600209156033091570340915803509186
:102290005903C701B6010E9467310E94293070932B
:1022A00099006093980080919504882309F433C1C4
:1022B000C0909004D0909104E0909204F090930428
:1022C00020E030E0A901C701B6010E946331181671
:1022D000D4F580918104909182048F3F2FEF920773
:1022E00029F001969093820480938104C701B6017E
:1022F0000E94F81320E030E040E051E40E94673192
:102300009B01AC0160E074E284E79BE40E94BC2F77
:102310006B017C010E9429307093970060939600B6
:10232000209156033091570340915803509159031F
:10233000C701B6010E9467310E942930709399004D
:102340006093980008C01092970010929600109227
:1023500099001092980060918A0470918B046F5FCD
:102360007F4F70938B0460938A0420919600309184
:10237000970080E090E0232BF1F0C0919600D0917F
:1023800097000E9455306B017C01BE0180E090E017
:102390000E9455309B01AC0160918C0470918D04BA
:1023A00080918E0490918F040E94BC2F20E03FEF1B
:1023B0004FE757E410C00E9455306B017C0120E0CC
:1023C00030EE4FEF54E460918C0470918D04809155
:1023D0008E0490918F040E9467319B01AC01C7016C
:1023E000B6010E94633187FD96C0809188048F5F9B
:1023F0008093880490E020916005309161058217F8
:102400009307A0F080916B05882319F0109288043F
:102410000DC0809171008D7F80937100809190003C
:102420008F7380939000109295047DC080918904F1
:10243000C0918804811128C0C0906505D0906605C0
:10244000E0906705F090680520E030E0A901C70141
:10245000B6010E9463311816BCF481E080938904B0
:10246000109290041092910410929204109293048E
:10247000C0928C04D0928D04E0928E04F0928F046E
:10248000C150C093880443C0109289041092820402
:1024900010928104E0916205F091630548E0C49FC9
:1024A000E00DF11D112480819181A281B38180937F
:1024B000900490939104A0939204B093930420E02D
:1024C00030E040E85EE364817581868197810E94F7
:1024D00067316B017C0180915A03682F70E080E0C6
:1024E00090E00E94553020E030E048EC52E40E9439
:1024F000BC2F9B01AC01C701B6010E9467316093FC
:102500008C0470938D0480938E0490938F041092AA
:102510008B0410928A048091640580FD04C010929F
:10252000950410929404FF91EF91DF91CF91BF91A8
:10253000AF919F918F917F916F915F914F913F915B
:102540002F91FF90EF90DF90CF90BF90AF909F9032
:102550008F907F906F905F904F900F900FBE0F9075
:102560001F901895CF92DF92EF92FF92CF93DF9357
:102570006B017C01EA0180918304811102C00E94F9
:10258000AD0E8091640580FF46C08091D204909189
:10259000D30408970CF03FC0809171008D7F809329
:1025A00071008091950481110E94C70E81E0809393
:1025B0009404109282041092810420E030E0A9017A
:1025C000C701B6010E9463311816DCF48091D20471
:1025D0009091D304FC01EE0FFF1FEE0FFF1FE65595
:1025E000FB4FC082D182E282F382FC01EE0FFF1F1B
:1025F000E656FB4FD183C08301969093D30480931A
:10260000D20480917100826080937100809190006B
:10261000806880939000DF91CF91FF90EF90DF90E2
:10262000CF9008958F929F92AF92BF92CF92DF92F8
:10263000EF92FF920F931F93CF93DF93EC017B01F7
:10264000D42E4801590180918304811102C00E9457
:10265000AD0E8091640580FF6BC0809171008D7F0D
:10266000809371008091940481110E94C70E81E0D3
:1026700080939504D0936305C0936205F092610541
:10268000E0926005D0926B05809265059092660598
:10269000A0926705B0926805109296041092970474
:1026A000109298041092990410928804888199815C
:1026B000AA81BB818093900490939104A09392048B
:1026C000B093930420E030E040E85EE36C817D81CC
:1026D0008E819F810E9467316B017C0180915A033A
:1026E000682F70E080E090E00E94553020E030E0FC
:1026F00048EC52E40E94BC2F9B01AC01C701B6011B
:102700000E94673160938C0470938D0480938E04D3
:1027100090938F0410928B0410928A048091710020
:102720008260809371008091900080688093900017
:10273000DF91CF911F910F91FF90EF90DF90CF909D
:10274000BF90AF909F908F900895809195040895C9
:102750008091640581700895809164058160809303
:1027600064050E948B2A0C94D507809164058E7FA6
:10277000809364050C948B2A6093560370935703DF
:102780008093580390935903089580935A030895B2
:1027900090915A03890F80935A03089590915A0398
:1027A000292F30E0281B31092A30310524F48AE032
:1027B00080935A030895981B90935A030895809329
:1027C000D40408958091D40490E0019666E070E00E
:1027D0000E9435338093D40408958091D40490E00E
:1027E000019766E070E00E9435338093D404089529
:1027F0008F929F92AF92BF92CF92DF92EF92FF9211
:102800000F931F93CF93DF936B017C01C0918104E1
:10281000D0918204BE0180E090E00E9455304B01CF
:102820005C01A701960160E070E08CE594E40E94F1
:10283000BC2F9B01AC01C501B4010E9467310E940D
:1028400029302091D404233009F473C028F42223C2
:1028500051F02130E9F02CC1243009F4A0C025301A
:1028600009F4E0C025C180E090E0A0E0BFE38093E0
:10287000560390935703A0935803B09359031092B3
:10288000840410928504109286041092870410C16B
:10289000109284041092850410928604109287048A
:1028A0006431710540F46A30710560F520E030E074
:1028B00040E85EE32BC0693C710508F0AAC080E0E7
:1028C00090E00E94553020E030E040EA51E40E9460
:1028D000532F20E030E044E353E40E94BC2F9B01DF
:1028E000AC010E94673120E030E040E05EE30E94EE
:1028F00067319B01AC0160E070E080E09EE30E94E4
:10290000532F44C020E030E040E05FE3C701B60150
:102910000E9467316B017C0180E090E0A0E0BEE3A3
:102920008093560390935703A0935803B093590391
:10293000BFC01092840410928504109286041092F5
:1029400087044AE0469F9001479F300D1124C9013A
:1029500068EB7BE00E942133BC016C5D754077FF22
:1029600003C0719561957109882777FD8095982F2F
:102970000E9457302EE333EC4EE259E30E94673158
:1029800020E030E040EC5EE30E94542F6093560359
:1029900070935703809358039093590389C0109202
:1029A0008404109285041092860410928704CE014C
:1029B00083709927892BE1F0BE016170772780E051
:1029C00090E00E94553020E030E040E05EE30E945D
:1029D000673120E030E040E45FE30E94542F6093D1
:1029E00056037093570380935803909359030CC078
:1029F00080E090E0A0E0BFE38093560390935703FC
:102A0000A0935803B0935903C770DD27CD2B09F06D
:102A10004FC0109256031092570310925803109211
:102A2000590346C0109284041092850410928604C3
:102A30001092870400E010E020E03FE3009356038B
:102A40001093570320935803309359036739710546
:102A500078F180E090E00E94553020E030E047E1DE
:102A600053E40E94532F20E030E04AE754E40E94F0
:102A7000BC2F20E030E048E452E40E94673120E0BF
:102A800030E040EA51E40E9499300E942430660F01
:102A9000771F660F771FFB01EA55FC4F20813181BC
:102AA00042815381C701B6010E9467316B017C01ED
:102AB000C701B601DF91CF911F910F91FF90EF9069
:102AC000DF90CF90BF90AF909F908F9008958091AE
:102AD000E5040895CF93DF9300D01F92CDB7DEB702
:102AE0009C0180917005843019F593E099833B83B4
:102AF0002A839093E9008FEF9091E800815095FD33
:102B000006C095ED9A95F1F700008111F5CF8091FF
:102B1000E80085FF0DC040E050E063E070E0CE01CA
:102B200001960E94CB178091E8008E778093E80091
:102B30000F900F900F90DF91CF910895CF93DF9377
:102B400000D01F92CDB7DEB720917005243021F55B
:102B500022E029839B838A8383E08093E9008FEFBF
:102B60009091E800815095FD06C095ED9A95F1F79A
:102B700000008111F5CF8091E80085FF0DC040E095
:102B800050E063E070E0CE0101960E94CB17809187
:102B9000E8008E778093E8000F900F900F90DF9100
:102BA000CF910895209170052430F1F422E0209314
:102BB000E9002FEF3091E800215035FD06C035EDDA
:102BC0003A95F1F700002111F5CF2091E80025FF9B
:102BD0000BC040E050E065E070E00E94CB178091B0
:102BE000E8008E778093E8000895CF93DF93EC019F
:102BF00090917005943009F046C080916503882358
:102C0000D9F0809166038823B9F09093E9008FEFA3
:102C10009091E800815095FD06C095E19A95F1F7F5
:102C200000008111F5CF8091E80085FF2CC040E0C5
:102C300050E060E170E017C081E08093E9008FEF21
:102C40009091E800815095FD06C095ED9A95F1F7B9
:102C500000008111F5CF8091E80085FF14C040E0AD
:102C600050E068E070E0CE010E94CB178091E80050
:102C70008E778093E80080E1FE01A5EDB4E001903D
:102C80000D928A95E1F7DF91CF91089580916F05BC
:102C9000811109C00E9460190E94BD198091E20053
:102CA00084608093E200089510926F05089508955E
:102CB00008950C94092842E061EC81E00E94DA1842
:102CC00042E061EC82E00E94DA1842E061EC83E0CD
:102CD0000E94DA1842E161EC84E00C94DA188091E9
:102CE0007205833009F455C030F4813071F08230C0
:102CF00009F48EC008958A3009F47AC08B3009F443
:102D000060C0893009F09CC020C080917105813A73
:102D100009F096C08091E800877F8093E800809159
:102D2000750590917605892B21F460E185ED94E09D
:102D300003C060E080E090E070E00E94161880918F
:102D4000E8008B778093E8000895809171058132C7
:102D500009F076C08091750590917605009719F07D
:102D6000039709F06DC08091E800877F8093E800A9
:102D70008091E80082FD05C0809170058111F8CF37
:102D80005FC08091F1008093E5048091E8008B772B
:102D900053C080917105813A09F052C08091750548
:102DA00090917605892B09F04BC08091E800877FD0
:102DB0008093E8008091E80080FFFCCF809165035C
:102DC00036C0809171058132D9F580917505909159
:102DD0007605892BA9F58091E800877F8093E8002C
:102DE0000E940F1980917305809365030C944A210A
:102DF00080917105813221F58091E800877F809371
:102E0000E8000E940F19809174058093E6040895EC
:102E100080917105813AA1F48091E800877F8093C9
:102E2000E8008091E80080FFFCCF8091E604809369
:102E3000F1008091E8008E778093E8000C940F19E0
:102E4000089584B7877F84BF88E10FB6F894809394
:102E50006000109260000FBE90E080E80FB6F8941A
:102E600080936100909361000FBE0E94B71C0E9486
:102E700060190E94BD198091E20084608093E20095
:102E800078940E94431C0E94B91C8BE593E00E9439
:102E90005E1C80917005853069F40E94CA2780917C
:102EA0006E058823B1F30E94F827882391F30E94CE
:102EB000B517EFCF0E94C11CECCF292F3327233049
:102EC0003105C9F064F42130310581F0223031053B
:102ED00009F043C08DE690E02CE837E042C0213293
:102EE0003105F1F02232310541F137C082E190E045
:102EF00029EF37E036C099278130910541F08230C3
:102F0000910541F0892B49F5E8E8F7E005C0EAE5CD
:102F1000F7E002C0E0E3F7E0849190E09F0121C078
:102F20006430D8F4E62FF0E0EE0FFF1FEE5FFB4FAA
:102F30002081318189E090E014C0643070F470E049
:102F4000FB01EE0FFF1FE650FC4F20813181FB019A
:102F5000EA50FC4F808190E004C080E090E020E0E7
:102F600030E0FA0131832083089580E189BD82E158
:102F700089BD09B400FEFDCF8091D8008F7D80937C
:102F8000D8008091E00082608093E0008091E000B2
:102F900081FDFCCF0895CF92DF92EF92FF920F93C5
:102FA0001F93CF93DF93EC018B016A010E942E19CE
:102FB000811133C0C114D10439F0F60180819181AF
:102FC000081B190BC80FD91FE12CF12C0115110595
:102FD00019F18091E80085FD16C08091E8008E7798
:102FE0008093E800C114D10449F0F60180819181F9
:102FF000E80EF91EF182E08285E00FC00E942E19D2
:10300000882321F30AC089918093F10001501109AE
:10301000FFEFEF1AFF0ADACF80E0DF91CF911F9127
:103020000F91FF90EF90DF90CF900895209177055A
:10303000309178052617370748F06115710539F486
:103040002091E8002E772093E80001C0B90140E00C
:1030500061157105A9F120917005222309F443C07F
:10306000253009F442C02091E80023FD40C02091A2
:10307000E80022FD32C02091E80020FFE9CF409116
:10308000F3002091F20030E0342BFC01CF016115F8
:10309000710559F02830310540F481918093F10099
:1030A000615071092F5F3F4FF1CF41E0283031056A
:1030B00009F040E02091E8002E772093E800C8CF87
:1030C0004111C9CF0AC080917005882361F0853015
:1030D00061F08091E80083FD0AC08091E80082FFE2
:1030E000F2CF80E0089582E0089583E0089581E0C2
:1030F000089520917705309178052617370748F015
:103100006115710539F42091E8002E772093E800CD
:1031100001C0B901FC0120E06115710591F18091B8
:103120007005882309F440C0853009F43FC08091C0
:10313000E80083FD3DC08091E80082FD2FC08091B2
:10314000E80080FFE9CF2091F3008091F20090E049
:10315000922B6115710559F08830910540F4249146
:103160002093F1003196615071090196F2CF21E070
:10317000089709F020E08091E8008E778093E800BE
:10318000CBCF2111CCCF0AC080917005882361F08C
:10319000853061F08091E80083FD0AC08091E800ED
:1031A00082FFF2CF80E0089582E0089583E00895E1
:1031B00081E00895982F973058F59093E90098177B
:1031C00039F07091EC002091ED005091F00003C0B7
:1031D000242F762F50E021FF19C03091EB003E7F65
:1031E0003093EB003091ED003D7F3093ED00309156
:1031F000EB0031603093EB007093EC002093ED0016
:103200005093F0002091EE0027FF07C09F5FD3CFBF
:103210008F708093E90081E0089580E008958091A7
:10322000710587FF11C08091E80082FD05C0809183
:1032300070058111F8CF11C08091E8008B770BC029
:1032400080917005882349F08091E80080FFF8CFD5
:103250008091E8008E778093E80008952091E40043
:103260003091E50095E64091EC00842F817040FF9D
:1032700022C08091E80080FD1CC0809170058823E9
:1032800091F0853091F08091EB0085FD10C0409168
:10329000E4005091E5004217530729F39A01915039
:1032A00011F784E0089582E0089583E0089581E0B5
:1032B000089580E008954091E80042FFDECF089530
:1032C0000E94CE190E94D619E0EEF0E08081816064
:1032D0008083E8EDF0E080818F77808319BCA7EDD3
:1032E000B0E08C918E7F8C9380818F7E8083109252
:1032F0006F0508950F931F93CF93DF930E94CE190C
:103300000E94D619C8EDD0E088818F7788838881A4
:103310008068888388818F7D888319BC10927005AE
:1033200010926C0510926E0510926D0500EE10E083
:10333000F80180818B7F808388818160888342E06F
:1033400060E080E00E94DA18E1EEF0E080818E7F9C
:103350008083E2EEF0E080818160808380818860FC
:103360008083F80180818E7F80838881806188835B
:10337000DF91CF911F910F910895E8EDF0E08081EA
:103380008F7E8083E7EDF0E080818160808384E040
:1033900082BF81E080936F050C947A19E8EDF0E02C
:1033A00080818E7F80831092E20008951092DA006F
:1033B0001092E10008951F920F920FB60F92112400
:1033C0002F933F934F935F936F937F938F939F932D
:1033D000AF93BF93EF93FF938091E10082FF0BC007
:1033E0008091E20082FF07C08091E1008B7F809393
:1033F000E1000E94421C8091DA0080FF1FC0809192
:10340000D80080FF1BC08091DA008E7F8093DA00A5
:103410008091D90080FF0DC080E189BD82E189BD26
:1034200009B400FEFDCF81E0809370050E9446162E
:1034300005C019BC109270050E9454168091E100DD
:1034400080FF19C08091E20080FF15C08091E200EA
:103450008E7F8093E2008091E20080618093E200A1
:103460008091D80080628093D80019BC85E0809359
:1034700070050E9458168091E10084FF30C0809151
:10348000E20084FF2CC080E189BD82E189BD09B4DE
:1034900000FEFDCF8091D8008F7D8093D800809171
:1034A000E1008F7E8093E1008091E2008F7E809327
:1034B000E2008091E20081608093E20080916C05DF
:1034C000882311F084E007C08091E30087FD02C0EB
:1034D00081E001C083E0809370050E9459168091BD
:1034E000E10083FF29C08091E20083FF25C0809125
:1034F000E100877F8093E10082E080937005109265
:103500006C058091E1008E7F8093E1008091E20064
:103510008E7F8093E2008091E20080618093E200E0
:1035200042E060E080E00E94DA188091F00088605C
:103530008093F0000E945716FF91EF91BF91AF91D9
:103540009F918F917F916F915F914F913F912F91BB
:103550000F900FBE0F901F9018951F920F920FB6ED
:103560000F9211242F933F934F935F936F937F9309
:103570008F939F93AF93BF93CF93DF93EF93FF937B
:10358000C091E900CF708091EC00D82FD17080FD00
:10359000D0E81092E9008091F000877F8093F000DE
:1035A00078940E94F11A1092E9008091F0008860EE
:1035B0008093F000CD2BCF70C093E900FF91EF9185
:1035C000DF91CF91BF91AF919F918F917F916F913B
:1035D0005F914F913F912F910F900FBE0F901F90D1
:1035E00018951F93CF93DF93CDB7DEB7AA970FB689
:1035F000F894DEBF0FBECDBFE1E7F5E088E08E0FA7
:103600009091F10091938E13FBCF0E946F168091E1
:10361000E80083FF1FC18091710590917205492FC9
:1036200050E04A30510508F015C1FA01E059FF4F4A
:103630000C944933803881F0823809F00BC18091B5
:1036400075058F708093E9008091EB0085FB8827DA
:1036500080F91092E90006C080916D0590916E0589
:10366000911182609091E800977F9093E800809399
:10367000F1001092F100C8C0282F2D7F09F0EAC098
:10368000882319F0823061F0E5C0809173058130A4
:1036900009F0E0C0933009F080E080936E052BC004
:1036A00080917305811127C0809175058F7009F491
:1036B000D1C08093E9002091EB0020FF1CC0933023
:1036C00021F48091EB00806214C09091EB00906136
:1036D0009093EB0021E030E0A90102C0440F551F98
:1036E0008A95E2F74093EA001092EA008091EB009D
:1036F00088608093EB001092E9008091E800877F5A
:1037000086C08111A7C0109173051F778091E300D7
:103710008078812B8093E3008091E800877F8093FD
:10372000E8000E940F198091E80080FFFCCF809193
:10373000E30080688093E300111102C082E001C0C1
:1037400083E08093700586C08058823008F082C084
:1037500080917305909174058C3D53E0950779F540
:1037600083E08A838AE289834FB7F894DE01139657
:1037700020E03EE051E2E32FF0E050935700E49167
:1037800020FF03C0E295EF703F5FEF708E2F90E057
:10379000EA3010F0C79601C0C0968D939D932F5FBD
:1037A000243149F74FBF8091E800877F8093E8007C
:1037B0006AE270E0CE0101960E94161814C0AE01B4
:1037C0004F5F5F4F609175050E945D17BC010097C8
:1037D00009F440C09091E800977F9093E8008981B8
:1037E0009A810E9479188091E8008B778093E80095
:1037F00031C0803879F58091E800877F8093E800B8
:1038000080916C058093F1008091E8008E77809321
:10381000E8000E940F191EC081111CC09091730511
:103820009230C0F48091E800877F8093E800909305
:103830006C050E940F1980916C05811106C0809162
:10384000E30087FD02C081E001C084E08093700541
:103850000E945B168091E80083FF0AC08091E80017
:10386000877F8093E8008091EB0080628093EB007B
:10387000AA960FB6F894DEBF0FBECDBFDF91CF91F1
:103880001F9108950895CF93809170058823A1F02A
:10389000C091E900CF709091EC00892F817090FD6C
:1038A00080E8C82B1092E9008091E80083FD0E9417
:1038B000F11ACF70C093E900CF9108959093EC0472
:1038C0008093EB0408958091EB049091EC040895AB
:1038D000E091EB04F091EC04309721F00190F0813D
:1038E000E02D099480E00895E091EB04F091EC0460
:1038F000309721F00280F381E02D09940895E09142
:10390000EB04F091EC04309721F00480F581E02D78
:10391000099408952091E9043091EA0482179307ED
:1039200071F09093EA048093E904E091EB04F09144
:10393000EC04309721F00680F781E02D099408957A
:103940002091E7043091E8048217930771F0909377
:10395000E8048093E704E091EB04F091EC043097E5
:1039600021F00084F185E02D0994089508950C94C8
:10397000B61C0E943D280E94DA0D0E9407290C9473
:10398000B82E5F926F927F928F929F92AF92BF926A
:10399000CF92DF92EF92FF920F931F93CF93DF931B
:1039A00000D000D01F92CDB7DEB70E941F0E98EF57
:1039B000C92E94E0D92E04E010E0AA24A394B12CDF
:1039C000502E802F0E948D0E4C01F6017290629055
:1039D0006F016826792661147104A1F40150110960
:1039E00078F78FEF89838A831B820E944628816043
:1039F000782F9D838C8349815A816B818D810E94B0
:103A0000711D38C080914D0581FD0E94960E2EE0FB
:103A100030E07501022E02C0EE0CFF1C0A94E2F7A2
:103A2000C70186219721892B09F129835A828E208B
:103A30009F2091E0892809F490E09B830E9446280A
:103A40008160782F9D838C8349815A816B818D8120
:103A50000E94711D000F111FF801E251FB4F808180
:103A60009181E826F926F182E08204C021503109D3
:103A700080F6B4CF0E940A2C1091ED040E94681CBD
:103A80001817D1F00E94681C8093ED040F900F90DE
:103A90000F900F900F90DF91CF911F910F91FF909A
:103AA000EF90DF90CF90BF90AF909F908F907F90DE
:103AB0006F905F900C94C40D0F900F900F900F902B
:103AC0000F90DF91CF911F910F91FF90EF90DF90BA
:103AD000CF90BF90AF909F908F907F906F905F90AE
:103AE0000895CF93DF93CDB7DEB72B970FB6F89439
:103AF000DEBF0FBECDBF4F83588769877A878B871C
:103B0000DE01119686E0FD0111928A95E9F785E0C4
:103B1000FE01379601900D928A95E1F749815A810D
:103B20006B817C818D819E810E94E8232B960FB64C
:103B3000F894DEBF0FBECDBFDF91CF910895CF9334
:103B4000882309F4C2C0C82F823859F40E94681C27
:103B500081FDBBC089E30E94C2260E948F2789E3B2
:103B60000CC0833879F40E94681C80FDAEC083E5E8
:103B70000E94C2260E948F2783E50E940427CF91CE
:103B80000C948F27843859F40E94681C82FD9DC0D4
:103B900087E40E94C2260E948F2787E4EECF8CEF35
:103BA0008C0F813A48F48C2F0E94202E81118DC0F9
:103BB0008C2F0E94C226E3CF80E28C0F883048F41D
:103BC000C77081E001C0880FCA95EAF70E944827B4
:103BD000D6CF8BE58C0F833078F4C53A29F0C63AFE
:103BE00031F083E890E005C081E890E002C082E80F
:103BF00090E0CF910C948A1C88E58C0F833108F0FB
:103C000064C0C83A39F1C93A41F1CA3A49F1CB3AEC
:103C100051F1CC3A59F1CD3A61F1C03B69F1CE3A5C
:103C200071F1CF3A79F1C13B81F1C23B89F1C33BDC
:103C300091F1C43B99F1C53BA1F1C63BA9F1C73B4A
:103C4000B1F1C83BB9F1C93BC1F1CA3BC9F180E050
:103C500090E038C082EE90E035C089EE90E032C04E
:103C60008AEE90E02FC085EB90E02CC086EB90E0D0
:103C700029C087EB90E026C08CEC90E023C08DEC4F
:103C800090E020C083E891E01DC08AE891E01AC06E
:103C900082E991E017C084E991E014C081E292E0EA
:103CA00011C083E292E00EC084E292E00BC085E294
:103CB00092E008C086E292E005C087E292E002C08E
:103CC0008AE292E0CF910C94A01CCF9108958823B2
:103CD00009F44BC0823859F40E94681C81FF45C02A
:103CE00089E30E94C2260E948F2789E30CC0833893
:103CF00071F40E94681C80FF38C083E50E94C226D0
:103D00000E948F2783E50E9404270C948F27843814
:103D100059F40E94681C82FF28C087E40E94C226D2
:103D20000E948F2787E4EFCF9CEF980F913A58F3CA
:103D300090E2980F983050F4877091E001C0990F8D
:103D40008A95EAF7892F0E944E27DFCF9BE5980FCF
:103D5000933020F480E090E00C948A1C885A8331E0
:103D600020F480E090E00C94A01C0895882321F0BA
:103D70000E9448270C948F270895882321F00E94E1
:103D80004E270C948F2708957F928F929F92AF9227
:103D9000BF92CF92DF92EF92FF920F931F93CF9338
:103DA000DF931F92CDB7DEB77C01C62E772EFC01C4
:103DB000058102950F70128111110E9465270E94E2
:103DC000BB26882379F0112369F080E28C0D8830BE
:103DD00048F082E00E94A4260E94BB2691E0D82EE3
:103DE000D92601C0D12CE72DE295EF70F0E0E6581E
:103DF000FF4F0C944933872D807F072D0F70882348
:103E000011F00295007F112389F0002309F499C174
:103E100080E28C0D883020F4802F0E94482703C058
:103E2000802F0E9458270E948F278BC18C2D0E94C3
:103E3000671E002309F4C3C180E28C0D883020F492
:103E4000802F0E944E2703C0802F0E945E270E9471
:103E50008F27B5C1872D807F972D9F70803211F4F9
:103E6000892F03C0892F8295807FCC2021F0F1E03B
:103E7000CF16A1F01DC0112339F0002319F1013034
:103E800009F50E9478279BC1002319F0013009F43D
:103E900096C189830E947B27898110C1112321F05B
:103EA000063008F08CC10EC0053008F088C106C18C
:103EB000112359F0002331F0F701958190FF41C1A2
:103EC0009F7095830E94B61E7AC1002309F4F6C044
:103ED0003EC1872D86958695837090E0009719F0F6
:103EE000019761F06CC1112321F08C2D972D9370F7
:103EF00002C080E090E00E948A1C61C1112321F081
:103F00008C2D972D937002C080E090E00E94A01C41
:103F100056C18C2D112319F00E94122B02C00E9451
:103F20007A2B0E94FF2B4BC1872D837009F052C062
:103F3000111145C18C2D829586958770880F880F49
:103F40009C2D9F70892E912CA12CB12C082E04C081
:103F5000880C991CAA1CBB1C0A94D2F7C4FE14C07E
:103F60000FE010E020E030E0B901A80104C0440FE8
:103F7000551F661F771F8A95D2F7CB01BA0160954E
:103F800070958095909503C060E070E0CB01272D7F
:103F900026952695237030E02230310569F02330D4
:103FA000310589F0682979298A299B292130310531
:103FB00071F00E94302503C1682979298A299B293B
:103FC0000E944C25FCC00E943025C501B4010E940E
:103FD0001425F5C0112319F0872D817001C0869535
:103FE000882309F4ECC08C2D829586958770880F04
:103FF000880F9C2D9F70892E912CA12CB12C082EFE
:1040000004C0880C991CAA1CBB1C0A94D2F7C4FEDD
:1040100014C00FE010E020E030E0B901A80104C0B6
:10402000440F551F661F771F8A95D2F7CB01BA013F
:10403000609570958095909503C060E070E0CB012D
:10404000272D269526952370422F50E042305105AA
:1040500069F04330510589F0682979298A299B291B
:104060004130510571F00E940A26A9C068297929BA
:104070008A299B290E942626A2C00E940A26C501E1
:10408000B4010E94EE259BC08C2D90E0FC01E05E07
:10409000F109E531F10508F050C0E657FF4F0C94E7
:1040A00049330C2D0F70872D8F71112321F00E9441
:1040B0008725802F07CF0E94A825802F0E94BD1E34
:1040C0007EC0112341F0053008F079C0872D8F7133
:1040D0000E94CD2574C0063008F071C0F7CF1123BF
:1040E00039F0872D8F710E94872569C01123C9F38C
:1040F000872D8F710E94A82562C0112329F0872D7A
:104100008F710E9472255BC00E94682558C01123E0
:1041100051F0172D1F71812F0E94872563E0812F99
:104120000E949B264CC081E00E94A426023008F425
:1041300046C082E00E94A42642C0112331F0002331
:1041400081F28C2D0E949F1D3AC0002389F28C2D94
:104150000E94671E34C0472D4F706C2DC7010E940E
:104160004A060E948C242BC0111129C0472D4F7084
:1041700050E042305105B9F04CF44115510581F041
:1041800041305105E1F40E94E02E19C04330510541
:1041900069F04430510599F48C2D0E94322F0FC0E4
:1041A0000E94C92E0CC00E94FC2E09C00E940F2F35
:1041B00006C0472D4F706C2DC7010E94650ADD2097
:1041C000F9F00E94972680FD1BC0F70112820E9421
:1041D00091260E948725C7010E940F210E949126E7
:1041E0000F90DF91CF911F910F91FF90EF90DF9093
:1041F000CF90BF90AF909F908F907F900C94A82508
:104200000F90DF91CF911F910F91FF90EF90DF9072
:10421000CF90BF90AF909F908F907F9008950F9315
:104220001F93CF93DF93EC01888199812B813C818F
:10423000232BB9F09F3F11F48F3F99F0CE010E94DC
:104240006408882371F0688179818A810E948D26B3
:104250008C010E9442260E940925B801CE010E94CD
:10426000C41EDF91CF911F910F9108950E94652781
:104270000E9475270E943A270E948F270E94B02C27
:104280000E94FF2B80E090E00E948A1C80E090E07A
:104290000C94A01C0E9455270C9436210E94822663
:1042A000292F22952F7030E02C3031054CF42A3024
:1042B00031056CF42250310922303105A8F407C0D1
:1042C0002C30310569F02F30310551F00DC0803FA1
:1042D00069F018F4803E40F409C0843F29F406C018
:1042E00093FB882780F9089580E0089581E0089580
:1042F000CF93DF9300D000D01F92CDB7DEB70F90E1
:104300000F900F900F900F90DF91CF910895CF9362
:10431000DF9300D000D000D0CDB7DEB726960FB621
:10432000F894DEBF0FBECDBFDF91CF9108951F93EC
:10433000CF93DF93C091F80416E08091F904C81779
:1043400099F0D0E01C9FF0011D9FF00D1124E65064
:10435000FB4F4081518162817381848195810E94EC
:1043600087212196C770E9CFDF91CF911F910895E2
:1043700040912A0550912B0560912C0570912D05D7
:1043800080912E0590912F050C94872180912F0507
:1043900082958F7009F054C080912C05882309F410
:1043A0004FC08091F804A091F90460912A057091A2
:1043B0002B0540912D0550912E05B6E08A1709F482
:1043C0003FC090E041155105C1F17F3F11F46F3FAF
:1043D000A1F1B89FF001B99FF00D1124E650FB4FF9
:1043E000218172132AC02081621327C022812111EA
:1043F00024C0238134812417350710F4215031095A
:10440000241B350B283C3105C0F420912F052F705B
:10441000206120932F0526E0289FF001299FF00DB1
:104420001124E150FB4F80818F70806180838AE28C
:1044300095E00E940F210C94972101968770BECFC2
:104440000895CF92DF92EF92FF920F931F93CF9335
:10445000DF93CDB7DEB762970FB6F894DEBF0FBE1D
:10446000CDBF8C0185E0F801DE011D9601900D9213
:104470008A95E1F7D8014C9111965C9111971296AB
:104480006C9112971396CD90DC90149730912A0579
:1044900070912B0580912D0590912E05009709F4C0
:1044A0006BC17F3F19F43F3F09F466C1E0902C05D2
:1044B000EE2009F4C0C020912F05C816D90628F0B7
:1044C000F601E81BF90BCF0104C0809590958C0D87
:1044D0009D1DFF24F394883C910578F0F12C207FFA
:1044E00009F0C6C07C2DD98AC88A89890E947821A2
:1044F0008AE295E00E940F21B1C0822F807F09F0EF
:1045000046C0751314C0341312C0611110C02F704F
:10451000206120932F050E94B8218AE295E00E9435
:104520000F2180912F05D80115968C932EC0CD2890
:1045300019F15F3F11F44F3FF9F0F62E61111CC0E5
:104540008091F8042091F90436E0821709F45AC0EA
:1045500090E0389FF001399FF00D1124E650FB4F99
:104560007181571306C07081471303C072817111A6
:1045700003C001968770E9CFF62E662309F418C1AF
:1045800080912F05816080932F05F12C11C1751347
:1045900008C0341306C0611104C080912F05D801F2
:1045A000C3C04D875E878D859E856A8B0E944E2194
:1045B0006A898823E1F16623D1F120912F05822FAA
:1045C00082958F7090E0029774F080912A05909107
:1045D0002B0598878F831986DB86CA862C87CE01A8
:1045E00007960E940F2186E0F801AAE2B5E001904B
:1045F0000D928A95E1F70E94C6210E94B821FF24FE
:10460000F394D6C04D875E878D859E850E94822655
:10461000292F22952F7030E0223031050CF0BCC0DC
:104620009F7009F0B6C0805E883008F4C1C0C80130
:104630000E940F21E4CFC816D90608F453C0F60132
:10464000E81BF90BCF01883C910508F450C0F12C10
:104650007C2DD98AC88A89890E947821EAE2F5E00E
:1046600086E0DF011D928A95E9F70E94B821A0C07B
:10467000751314C0341312C0611110C080912F053E
:10468000F8018583C8010E940F2186E0EAE2F5E087
:10469000DF011D928A95E9F7FE2C8AC04D875E875F
:1046A0008D859E856A8B0E944E216A89882309F434
:1046B000BECF662309F4BBCF20912F05822F8295B0
:1046C0008F7090E002970CF48ECF80912A05909124
:1046D0002B059A8389831B82DD82CC822E83CE01B7
:1046E00001967FCF809590958C0D9D1DACCFF62EB9
:1046F000662309F49CCF75132EC034132CC020916F
:104700002F0520FD1FC0822F82958F70D9F0D80110
:1047100015962C9315978F3049F08F5F982F9295AF
:10472000907F822F8F70892B15968C93C8010E94E1
:104730000F2186E0F801AAE2B5E001900D928A957A
:10474000E1F793CF86E0F801AAE2B5E001900D927F
:104750008A95E1F72DC04D875E878D859E850E94E5
:104760004E21811140CF80912F05816080932F05CC
:10477000C8010E940F211CC0662309F458CF4D8741
:104780005E878D859E850E944E21882309F44FCF38
:104790002ACF811148CF0CC0243031050CF047CF0F
:1047A0009F7009F440CFF8019581907F09F03BCFCD
:1047B0008F2D62960FB6F894DEBF0FBECDBFDF918E
:1047C000CF911F910F91FF90EF90DF90CF900895C0
:1047D0001F93CF93DF93CDB7DEB72C970FB6F89426
:1047E000DEBF0FBECDBF4F83588769877A878B871F
:1047F0009C87CE0107960E942122882369F08F8131
:1048000098852A853B85232BF1F19F3F09F063C0F2
:104810008F3F09F060C037C086E0FE013796DE01A9
:10482000119601900D928A95E1F76F817885EA855E
:10483000FB85309741F17F3F11F46F3F21F12091CB
:10484000F90430E0C9010196877099274091F80476
:1048500050E08417950709F447C069837A83FD8384
:10486000EC8396E0929FD001939FB00D1124A65047
:10487000BB4FFE01319601900D929A95E1F780931E
:10488000F9040E94972116E08091F8049091F904B0
:104890008917C1F1189FC001112486509B4F0E94B7
:1048A0002122882379F1E091F8041E9FF001112460
:1048B000E650FB4F408151816281738184819581F3
:1048C0000E9487218091F80490E0019687709927D3
:1048D0008093F804D9CF4F81588569857A858B8577
:1048E0009C850E948721CFCF0E944A211092F90413
:1048F0001092F804EAE2F5E086E0DF011D928A9565
:10490000E9F7C1CF2C960FB6F894DEBF0FBECDBF2E
:10491000DF91CF911F910895EF92FF920F931F9314
:10492000CF93DF938C01009709F46CC0F12CEE2437
:10493000E394E8012196F8018491843740F48430AF
:1049400008F051C0813081F0823019F15BC08537A9
:1049500009F444C0A8F19CE7980F903708F052C0C2
:104960008F770E94671E41C00E5F1F4FFE01C491EA
:1049700080E28C0F883048F4C7708E2D01C0880FFC
:10498000CA95EAF70E94682714C08C2F0E949F1DC9
:104990002DC00E5F1F4FFE01C49180E28C0F883046
:1049A00058F4C7708E2D01C0880FCA95EAF70E948F
:1049B0006E270E948F271AC08C2F0E94671E16C078
:1049C0000E5F1F4FFE01C491CC2381F08FE99FE061
:1049D0000197F1F700C00000C150F6CF0E5F1F4FE6
:1049E000FE01F49003C00E949F1D8E018F2D88232D
:1049F00009F49FCFEFE9FFE03197F1F700C0000025
:104A00008150F5CFDF91CF911F910F91FF90EF90E3
:104A100008950895609334057093350580933605A5
:104A2000909337050C9436210F931F930091340512
:104A3000109135052091360530913705DC01CB0109
:104A4000802B912BA22BB32B8093340590933505AB
:104A5000A0933605B09337051F910F910C94362122
:104A60000F931F9300913405109135052091360561
:104A700030913705DC01CB0180239123A223B3239E
:104A80008093340590933505A0933605B093370590
:104A90001F910F910C9436210F931F9300913405B1
:104AA000109135052091360530913705DC01CB0199
:104AB00080279127A227B32780933405909335054B
:104AC000A0933605B09337051F910F910C943621B2
:104AD0001092300510923105109232051092330574
:104AE0000C94362141E050E060E070E004C0440FD7
:104AF000551F661F771F8A95D2F740933005509354
:104B0000310560933205709333050C94362141E0F2
:104B100050E060E070E004C0440F551F661F771F2F
:104B20008A95D2F78091300590913105A091320598
:104B3000B0913305482B592B6A2B7B2B40933005C2
:104B40005093310560933205709333050C943621F0
:104B500041E050E060E070E004C0440F551F661F64
:104B6000771F8A95D2F74095509560957095809102
:104B7000300590913105A0913205B091330548235D
:104B800059236A237B23409330055093310560936A
:104B90003205709333050C94362141E050E060E01B
:104BA00070E004C0440F551F661F771F8A95D2F727
:104BB0008091300590913105A0913205B091330577
:104BC000482759276A277B274093300550933105A2
:104BD00060933205709333050C9436210F931F9325
:104BE0000091300510913105209132053091330547
:104BF000DC01CB01802B912BA22BB32B80933005B2
:104C000090933105A0933205B09333051F910F9116
:104C10000C9436210F931F930091300510913105AC
:104C20002091320530913305DC01CB0180239123A3
:104C3000A223B3238093300590933105A0933205CE
:104C4000B09333051F910F910C9436210F931F934E
:104C500000913005109131052091320530913305D6
:104C6000DC01CB0180279127A227B3278093300551
:104C700090933105A0933205B09333051F910F91A6
:104C80000C9436210895CF92DF92EF92FF920F930A
:104C90001F93CF93DF938C01C0903405D0903505DE
:104CA000E0903605F0903705809130059091310500
:104CB000A0913205B0913305C82AD92AEA2AFB2AE5
:104CC000CFE1D0E0D701C6010C2E04C0B695A79560
:104CD000979587950A94D2F780FF06C0B8018C2F6C
:104CE0000E94EA0C019721F4219760F780E001C04F
:104CF0008C2FDF91CF911F910F91FF90EF90DF905C
:104D0000CF900895CF93DF93EC010E944326BE011C
:104D10000E94EA0CDF91CF910895CB010E94822678
:104D2000089580913805859585958595089580919C
:104D300038058770089598E0899F90011124262BEB
:104D4000209338050C94872520913805809582237F
:104D500080933805982F977069F430E0482F5527D5
:104D600047FD50952417350729F08595859585953C
:104D70000C94A825089590913805977081E009F466
:104D800080E0089590916503992321F09091660346
:104D9000911109C02091670330916803F90132969F
:104DA0009FEF40E01FC0982F9695969596959F305F
:104DB00050F5E0916703F0916803E90FF11D8770EA
:104DC00021E030E0A90102C0440F551F8A95E2F7A7
:104DD000CA019181892B818308959F3F39F04F5FEC
:104DE0004E3041F051915813F8CF0DC05111F7CF0B
:104DF000942FF5CF9F3F39F0F901E90FF11D97FD91
:104E0000FA9582830895089590916503992321F07E
:104E100090916603911109C0209167033091680356
:104E2000F9013296205F3F4F1FC0982F96959695B7
:104E300096959F30F0F4E0916703F0916803E90FD5
:104E4000F11D877021E030E0A90102C0440F551F19
:104E50008A95E2F7CA01809591818923818308951B
:104E60003196E217F30729F090819813F9CF108259
:104E7000F7CF089581E090E0E0916703F091680337
:104E8000E80FF91F1082019680319105A9F7089566
:104E900090914C05892B80934C05089580959091B5
:104EA0004C05892380934C05089510924C05089574
:104EB00090914B05892B80934B0508958095909197
:104EC0004B05892380934B05089510924B05089557
:104ED00090914A05892B80934A0508958095909179
:104EE0004A05892380934A05089510924A0508953A
:104EF00080933905089510923905089580916703CC
:104F000090916803FC0131969C01205F3F4F80E047
:104F1000919191118F5FE217F307D1F70895E09116
:104F20006703F091680380914C058083E0916703EB
:104F3000F0916803908180914B05892B8083E091EB
:104F40006703F0916803908180914A05892B8083E3
:104F500080913905882361F0E0916703F09168033F
:104F60009081892B80830E947E27811110923905C0
:104F700080916703909168030C94741C20E0009763
:104F800039F0AC0141505109842395232F5FF7CFAD
:104F9000822F089580917005843039F110924E056A
:104FA00020E488E190E00FB6F894A8958093600023
:104FB0000FBE2093600080E00E942A0580E00E94DE
:104FC000C40D83B7817F846083BF83B7816083BF53
:104FD0007894889583B78E7F83BF88E10FB6F89465
:104FE00080936000109260000FBE089508950895A8
:104FF00080E00E942A050E94F6270E941F0E0E9450
:10500000F7270E94970E91E0811101C090E0892F4F
:1050100008950E944A2180E00E942A050E94B82E2D
:105020000E94681C0C94C40D1F920F920FB60F9231
:1050300011248F939F93AF93BF9380914E0581115D
:1050400013C080914F0590915005A0915105B091EA
:1050500052054196A11DB11D80934F0590935005B7
:10506000A0935105B0935205BF91AF919F918F913D
:105070000F900FBE0F901F90189582E084BD93E0B3
:1050800095BD9AEF97BD80936E0008952FB7F89461
:1050900080914F0590915005A0915105B091520516
:1050A0002FBF0895CF92DF92EF92FF920F931F933D
:1050B0002FB7F89440914F055091500560915105DC
:1050C000709152052FBF6A017B01EE24FF248C01F1
:1050D00020E030E0C016D106E206F30610F441509D
:1050E00051099A01281B390BC9011F910F91FF909B
:1050F000EF90DF90CF9008951F920F920FB60F920E
:1051000011248F939F93AF93BF9380914F059091FC
:105110005005A0915105B09152050196A11DB11DF8
:1051200080934F0590935005A0935105B09352057D
:10513000BF91AF919F918F910F900FBE0F901F90D5
:1051400018950E946019F8942FEF87EA91E6215094
:1051500080409040E1F700C0000087E090EBDC0168
:1051600080937B0590937C05A0937D05B0937E058D
:105170009CE088E10FB6F894A895809360000FBE7C
:1051800090936000FFCFCF92DF92EF92FF920F9348
:105190001F93CF93DF93D82FC4E0EE24E394F12C38
:1051A0008C2F0E948D0E6C010EE010E09701002EF6
:1051B00002C0220F331F0A94E2F72C213D21232B3A
:1051C00049F0602F7C2F80E00E94660AD81302C04D
:1051D00081E006C00150110948F7C15008F780E08E
:1051E000DF91CF911F910F91FF90EF90DF90CF90C3
:1051F0000895CF93C82F8CE20E94C328882321F002
:105200008C2FCF910C94C32880E0CF910895CF9339
:105210000E94582A811102C00E94342AC5E6C1505A
:1052200049F00E941F0E8FE39CE90197F1F700C03F
:105230000000F5CF89E20E94F928811113C18AE2AA
:105240000E94F92881110E94342A85E00E94F928E1
:1052500081110E94A1280E94632A80934D0587E056
:105260000E94F9288823A9F18BE10E94F92888235C
:1052700051F080914D0581FB222720F991E0922782
:1052800090FB81F90EC08EE00E94F928882361F01E
:1052900080914D0582FB222720F991E0922790FB17
:1052A00082F980934D0515C080E10E94F928909104
:1052B0004D05882341F093FB222720F981E08227C6
:1052C00080FB93F904C0892F809580FB90F990931F
:1052D0004D0580914D050E94672A0E94752A809392
:1052E000790580EE0E94F928882341F080917905A4
:1052F000982F909590FB80F98093790589E30E941F
:10530000F928882359F08091790581FB222720F91B
:1053100091E0922790FB81F98093790582EE0E94BB
:10532000F928882359F08091790582FB222720F9FA
:1053300091E0922790FB82F98093790586EE0E9496
:10534000F928882359F08091790583FB222720F9D9
:1053500091E0922790FB83F98093790583EE0E9478
:10536000F928882359F08091790584FB222720F9B8
:1053700091E0922790FB84F98093790585E30E9460
:10538000F928882359F08091790585FB222720F997
:1053900091E0922790FB85F98093790581E30E9443
:1053A000F928882359F08091790586FB222720F976
:1053B00091E0922790FB86F98093790581E10E9424
:1053C000F928882359F08091790587FB222720F955
:1053D00091E0922790FB87F9809379058091790578
:1053E0000E94792A8091790587FB882780F980932C
:1053F000660387E20E94F928C82F8EE10E94F928EF
:105400008111C2608FE10E94F9288111C46080E29D
:105410000E94F9288111C86081E20E94F928811157
:10542000C06182E20E94F9288111C06283E20E9479
:10543000F9288111C06484E20E94F928882311F0C0
:10544000C06802C0CC2329F08C2F0E94702A6C2FD8
:1054500003C00E946C2A682F70E080E090E0CF913A
:105460000C940A25CF9108956DEE7EEF80E090E0D8
:105470000E946F3360E082E090E00E945D3360E064
:1054800083E090E00E945D3360E084E090E00E9461
:105490005D3360E085E090E00E945D3360E086E08F
:1054A00090E00E945D336FEF87E090E00C945D33F5
:1054B00080E090E00E94573321E08D3E9E4F09F03E
:1054C00020E0822F089582E090E00C944F33682F03
:1054D00082E090E00C945D3383E090E00C944F33D5
:1054E000682F83E090E00C945D3384E090E00C94AE
:1054F0004F33682F84E090E00C945D3386E090E0B9
:105500000C944F33682F86E090E00C945D3387E075
:1055100090E00C944F33682F87E090E00C945D335B
:105520008091550580FF0BC060916C0385E0689FFA
:10553000B001112475956795759567952BC081FF0E
:1055400009C060916C0385E0689FB00111247595D6
:10555000679520C082FF07C060916C0385E0689F5B
:10556000B001112417C0909156059923D1F0609194
:105570006B03961788F720916C0385E0289F9001B4
:105580001124929FA001939F500D112470E0CA0135
:105590000E9435336038710540F46115710539F0AA
:1055A00002C065E070E0862F08958FE7089581E0DE
:1055B00008958091550580FF08C060916A0370E0EE
:1055C000759567957595679521C081FF06C06091B7
:1055D0006A0370E07595679519C082FF04C06091F9
:1055E0006A0370E010C0909156059923C1F0609154
:1055F00069039617A0F780916A03899FC00111245F
:1056000070E00E9435336038710528F4611571052A
:1056100021F0862F08958FE7089581E0089561E0D5
:1056200070E0F4CF803F21F40E94902A819504C05D
:10563000813F29F40E94902A809359050895823F62
:1056400021F40E94902A819504C0833F29F40E948E
:10565000902A809358050895893F19F40E94D92A09
:1056600005C08A3F31F40E94D92A819580935A055A
:1056700008958B3F21F40E94D92A819504C08C3F64
:1056800029F40E94D92A80935B050895843F21F470
:1056900080915705816017C0853F21F4809157059F
:1056A000826011C0863F21F48091570584600BC051
:1056B000873F21F480915705886005C0883F31F409
:1056C0008091570580618093570508958D3F21F49F
:1056D0008091550581600BC08E3F21F48091550566
:1056E000826005C08F3F29F48091550584608093C6
:1056F00055050895803F39F48091590587FF6CC0A6
:105700001092590569C0813F29F4809159051816F6
:10571000BCF362C090915805823F29F497FF5CC0AA
:105720001092580559C0833F19F41916CCF354C090
:10573000893F41F480915A0518160CF04DC0109223
:105740005A054AC08A3F29F480915A0587FF44C010
:10575000F6CF8B3F39F480915B0587FF3DC01092F7
:105760005B053AC08C3F29F480915B051816BCF3A9
:1057700033C0843F21F4809157058E7F17C0853F49
:1057800021F4809157058D7F11C0863F21F48091CF
:1057900057058B7F0BC0873F21F480915705877F8A
:1057A00005C0883F31F4809157058F7E809357055F
:1057B00013C08D3F21F4809155058E7F0BC08E3F25
:1057C00021F4809155058D7F05C08F3F29F480918C
:1057D00055058B7F809355058091580581110EC02A
:1057E0008091590581110AC080915A05811106C026
:1057F00080915B05811102C010925605089587E5DE
:1058000095E00E947F1C0E94462890935405809347
:10581000530508951F93CF93DF9380915305909183
:1058200054050E945228AC0190915605992321F00D
:1058300020916D0330E006C020916E038AE0289F1E
:10584000900111244217530708F486C0809158052F
:10585000C0915905D0915A0510915B05811107C07F
:10586000C11176C0D11174C0111172C075C09F3FB3
:1058700019F09F5F90935605181624F40E94902A01
:10588000809358058091580587FF05C00E94902A93
:105890008195809358051C1624F40E94902A8093C9
:1058A00059058091590587FF05C00E94902A81956E
:1058B0008093590560915805662339F1C0915905C7
:1058C000CC2319F1772767FD7095872F972F0E94BA
:1058D000573023E333E343E35FE30E9467310E94E1
:1058E0002430609358056C2F772767FD7095872FBC
:1058F000972F0E94573023E333E343E35FE30E9493
:1059000067310E942430609359051D1624F40E94CB
:10591000D92A80935A0580915A0587FF05C00E94B5
:10592000D92A819580935A05111624F40E94D92A08
:1059300080935B0580915B0587FF05C00E94D92A93
:10594000819580935B05DF91CF911F910C94FF2B84
:105950009F3F09F08ECF96CFDF91CF911F91089591
:10596000E7E5F5E085E0DF011D928A95E9F7109201
:105970005605109255050895833081F128F4813041
:1059800059F08230D1F00895853009F449C0B8F15A
:10599000863009F456C0089580916E03262F30E0BA
:1059A000280F311D2F3F310524F4680F60936E03DB
:1059B00008958FEF80936E03089580916D03262FD5
:1059C00030E0280F311D2F3F310524F4680F60931C
:1059D0006D0308958FEF80936D03089580916C039C
:1059E000262F30E0280F311D2F3F310524F4680F9A
:1059F00060936C0308958FEF80936C0308958091FA
:105A00006B03262F30E0280F311D2F3F310524F482
:105A1000680F60936B0308958FEF80936B03089575
:105A200080916A03262F30E0280F311D2F3F31056A
:105A300024F4680F60936A0308958FEF80936A03DC
:105A4000089580916903262F30E0280F311D2F3FE4
:105A5000310524F4680F6093690308958FEF8093F4
:105A600069030895833011F128F4813049F08230C0
:105A700091F00895853081F120F18630C1F10895CB
:105A800080916E03681720F4861B80936E0308953F
:105A900010926E03089580916D03681720F4861BA1
:105AA00080936D03089510926D03089580916C03A7
:105AB000681720F4861B80936C03089510926C0382
:105AC000089580916B03681720F4861B80936B0305
:105AD000089510926B03089580916A03681720F46B
:105AE000861B80936A03089510926A03089580913B
:105AF0006903681720F4861B809369030895109248
:105B0000690308950F931F93482F50E0FA013597CA
:105B1000EF33F10508F08CC0E156FF4F0C94493388
:105B20000E94631C892B59F00E94631C90935D05B1
:105B300080935C050E944A2180E090E004C080913F
:105B40005C0590915D050E945E1C6BC080914D05C7
:105B5000817F8E7F80934D0581E080935F0569C0D2
:105B60000E944A210E94C70E0E94BB070E94A128E2
:105B700058C090914D05892F8095817080FB90F9D8
:105B800029F09660986090934D0553C0997F977F58
:105B900090934D0546C080914D0581FB222720F949
:105BA00091E0922790FB81F980934D059923C9F1EB
:105BB00080914D05816080934D0533C080914D05E6
:105BC00082FB222720F991E0922790FB82F9ECCF0B
:105BD00080914D0583FB222720F991E0922790FBCD
:105BE00083F9E2CF0E944A219091660381E08927E0
:105BF0008093660316C0895301C08D5141E050E087
:105C000060E070E08A019B0104C0000F111F221F99
:105C1000331F8A95D2F7C901B8010E940A250E9454
:105C20004A2181E006C061E070E080E090E0F5CFBD
:105C300080E01F910F91089580E0089580E008951D
:105C4000CF93C82F80915F05813069F018F08230C2
:105C5000C9F184C0E0916703F091680380818232CA
:105C600009F07EC007C0E0916703F091680380816E
:105C7000823261F48C2F0E941C2E811104C08C2F63
:105C80000E94822D1DC081E090E01AC08C2F0E94DE
:105C90001E2E811114C0C43179F048F4CB3079F054
:105CA000C03109F061C082E080935F0508C0C9324D
:105CB00019F0C83321F058C010925F0555C081E03B
:105CC000817054C0C93291F120F5C43179F1B0F43A
:105CD000C73009F047C08EE180936E0382E3809362
:105CE0006D038AE080936C0384E180936B0388E00A
:105CF00080936A0388E28093690334C0CE51C63032
:105D000088F5EC2FF0E0E65FFB4F808180935E0525
:105D100029C0CE34E9F020F4CB3421F56AE013C079
:105D2000C13579F0C235F1F461E00DC080915E05B6
:105D3000882319F010925E0515C081E080935F05FD
:105D400015C061E006C080915E050E94BC2C0AC0AF
:105D50006AE080915E050E94322D04C010925F05BA
:105D600080E004C081E002C080E0AACFCF91089516
:105D70000E94582A811102C00E94342A0E947E2A61
:105D800080937A0580FF02C0869501C080E00C9464
:105D90002A0580917A05982F9695292F30E0233097
:105DA00031054CF49F5F990F8170892B816080933E
:105DB0007A050E94822A80917A0586950C942A059C
:105DC00080917A05982F969591F09158990F81704E
:105DD000892B80937A058E7F91E009F490E0809181
:105DE0007A0590FB80F980937A050E94822A80913F
:105DF0007A0586950C942A0580917A05982F9095BE
:105E000090FB80F980937A050E94822A80917A051E
:105E100080FF02C0869501C080E00C942A05909115
:105E20007A05892F86958F5F8F779170843028F45B
:105E3000880F892B80937A0502C090937A05809110
:105E40007A058E7F91E009F490E080917A0590FBCD
:105E500080F980937A050E94822A80917A0586953E
:105E60000C942A0520917A05922F96958927982FD0
:105E7000990F822F8170892B80937A058E7F91E014
:105E800009F490E080917A0590FB80F980937A057F
:105E90000E94822A80917A0586950C942A05809129
:105EA0007A05869508955058BB27AA270ED0D1C1F0
:105EB000C2D130F0C7D120F031F49F3F11F41EF46D
:105EC000B7C10EF4E095E7FB9FC1E92FD3D180F372
:105ED000BA17620773078407950718F071F49EF5E7
:105EE000EBC10EF4E0950B2EBA2FA02D0B01B901DA
:105EF00090010C01CA01A0011124FF27591B99F040
:105F0000593F50F4503E68F11A16F040A22F232F4B
:105F1000342F4427585FF3CF469537952795A7959B
:105F2000F0405395C9F77EF41F16BA0B620B730B42
:105F3000840BBAF09150A1F0FF0FBB1F661F771FB3
:105F4000881FC2F70EC0BA0F621F731F841F48F468
:105F5000879577956795B795F7959E3F08F0B3CFEE
:105F60009395880F08F09927EE0F979587950895D8
:105F700027D108F481E008950CD06BC163D140F0C3
:105F80005AD130F021F45F3F19F03EC1511195C153
:105F90004FC170D198F39923C9F35523B1F3951BE1
:105FA000550BBB27AA2762177307840738F09F5F3A
:105FB0005F4F220F331F441FAA1FA9F333D00E2EA9
:105FC0003AF0E0E830D091505040E695001CCAF716
:105FD00029D0FE2F27D0660F771F881FBB1F2617DB
:105FE00037074807AB07B0E809F0BB0B802DBF01AE
:105FF000FF2793585F4F2AF09E3F510568F004C178
:106000005CC15F3FECF3983EDCF38695779567952E
:10601000B795F7959F5FC9F7880F911D969587955E
:1060200097F90895E1E0660F771F881FBB1F62177D
:1060300073078407BA0720F0621B730B840BBA0B3B
:10604000EE1F88F7E095089504D06894B11135C12A
:10605000089518D188F09F5790F0B92F9927B7511C
:10606000A0F0D1F0660F771F881F991F1AF0BA951C
:10607000C9F712C0B13081F01FD1B1E008951CC141
:10608000672F782F8827B85F39F0B93FCCF3869512
:1060900077956795B395D9F73EF49095809570956F
:1060A00061957F4F8F4F9F4F0895E89409C097FBEC
:1060B0003EF490958095709561957F4F8F4F9F4FDF
:1060C0009923A9F0F92F96E9BB279395F695879523
:1060D00077956795B795F111F8CFFAF4BB0F11F4E6
:1060E00060FF1BC06F5F7F4F8F4F9F4F16C088238D
:1060F00011F096E911C0772321F09EE8872F762FC3
:1061000005C0662371F096E8862F70E060E02AF003
:106110009A95660F771F881FDAF7880F96958795EF
:1061200097F9089588D018F011F08CD038F480C019
:10613000C4C0E92F9FD0B0F35523C9F3E7FB621722
:10614000730784079507A8F199F3E92FFF278823A0
:106150002AF03197660F771F881FDAF7952F55279A
:10616000442332F091505040220F331F441FD2F786
:10617000BB27E91BF50B621B730B840BB109C1F242
:1061800022F4620F731F841FB11D31972AF0660F2E
:10619000771F881FBB1FEFCF915050405AF041F03E
:1061A000882332F0660F771F881F91505040C1F747
:1061B000939530C08695779567959F5FD9F7F8CF0F
:1061C000990F0008550FAA0BE0E8FEEF1616170608
:1061D000E807F907C0F012161306E407F50798F070
:1061E000621B730B840B950B39F40A2661F0232B89
:1061F000242B252B21F408950A2609F4A140A69505
:106200008FEF811D811D089597F99F6780E870E0E9
:1062100060E008959F3F31F0915020F48795779585
:106220006795B795880F911D9695879597F908956D
:106230009FEF80EC089500240A941616170618069E
:106240000906089500240A9412161306140605067A
:106250000895092E0394000C11F4882352F0BB0F0B
:1062600040F4BF2B11F460FF04C06F5F7F4F8F4F6E
:106270009F4F089557FD9058440F551F59F05F3FA9
:1062800071F04795880F97FB991F61F09F3F79F058
:1062900087950895121613061406551FF2CF4695DA
:1062A000F1DF08C0161617061806991FF1CF86955C
:1062B0007105610508940895E894BB276627772740
:1062C000CB0197F908957CDF08F48FEF08950BD088
:1062D000C0CFB1DF28F0B6DF18F0952309F094CFD6
:1062E000A7CF1124EACFC6DFA0F3959FD1F3950F76
:1062F00050E0551F629FF001729FBB27F00DB11D4A
:10630000639FAA27F00DB11DAA1F649F6627B00DD9
:10631000A11D661F829F2227B00DA11D621F739FC2
:10632000B00DA11D621F839FA00D611D221F749FD0
:106330003327A00D611D231F849F600D211D822F17
:10634000762F6A2F11249F5750408AF0E1F088235E
:106350004AF0EE0FFF1FBB1F661F771F881F91506B
:106360005040A9F79E3F510570F04ECFA6CF5F3F3A
:10637000ECF3983EDCF3869577956795B795F7959E
:10638000E7959F5FC1F7FE2B880F911D9695879526
:1063900097F90895FA01EE0FFF1F30962105310598
:1063A00099F16115710561F48038BFE39B0749F1EC
:1063B00068949038810561F08038BFEF9B0741F009
:1063C000992342F5FF3FE1053105210511F1E894DC
:1063D0000894E795D901AA2329F4AB2FBE2FF85FC3
:1063E000D0F310C0FF5F70F4A695E0F7F73950F0D6
:1063F00019F0FF3A38F49F779F930CD00F9007FC69
:10640000905808953EF014CF60E070E080E89FE37C
:1064100008954FE79F775F934F933F932F939ED0BD
:106420002F913F914F915F9152DF05C019F40EF00B
:10643000EBCE42CFFDCE26DFC8F39638C0F707F883
:106440000F92E8942BE33AEA48EB5FE74EDF0F92B6
:106450000F920F924DB75EB70F92C0D0ECEBF1E008
:1064600016D04F915F91EF91FF91E595EE1FFF1FC1
:1064700049F0FE57E0684427EE0F441FFA95E1F714
:106480004195550B32D00F9007FE26C00895DF933B
:10649000CF931F930F93FF92EF92DF927B018C01BA
:1064A000689405C0DA2EEF011EDFFE01E894A59185
:1064B0002591359145915591AEF3EF0106DDFE0131
:1064C0009701A801DA9479F7DF90EF90FF900F9190
:1064D0001F91CF91DF9108959B01AC0160E070E0C6
:1064E00080E89FE349CD90CE95CECCDEE8F39923AA
:1064F000D9F3940F511DBBF39150504094F059F0D3
:10650000882332F0660F771F881F91505040C1F7E3
:106510009E3F510544F7880F911D9695879597F9F1
:1065200008955F3FACF0983E9CF0BB278695779529
:106530006795B79508F4B1609395C1F7BB0F58F70D
:1065400011F460FFE8CF6F5F7F4F8F4F9F4FE3CF16
:10655000B4CE0EF05FCE6CCE689456CE93DEC8F308
:106560009923D1F3C6F3DF93CF931F930F93FF9239
:10657000C92FDD2788232AF02197660F771F881FF0
:10658000DAF720E030E040E85FEB9FE3883920F065
:10659000803E30F021968F7787DCE4EEF1E003C097
:1065A00083DCE1E1F2E073DF8B01BE01EC01FB2E45
:1065B0006F5771097595771F880B990B78DD28E166
:1065C00032E741E35FE38FDEAF2D9801AE01FF902C
:1065D0000F911F91CF91DF9178DC3BCEFA01DC0166
:1065E000AA0FBB1F9B01AC01BF5728F422273327FA
:1065F000442750781FC0B75188F4AB2F002446952C
:1066000037952795011CA395D2F3002069F0220F3E
:10661000331F441FB395DAF30DD045CC61307105BB
:10662000A0E88A07B94630F49B01AC0166277727BA
:1066300088279078309621F02083318342835383DA
:106640000895AA1BBB1B51E107C0AA1FBB1FA617B9
:10665000B70710F0A61BB70B881F991F5A95A9F70B
:1066600080959095BC01CD01089597FB072E16F4F7
:10667000009407D077FD09D00E94213307FC05D094
:106680003EF4909581959F4F0895709561957F4F49
:106690000895EE0FFF1F0590F491E02D0994F999EC
:1066A000FECF92BD81BDF89A992780B50895A8E1E3
:1066B000B0E042E050E00C947733262FF999FECFFA
:1066C00092BD81BDF89A019700B4021639F01FBA45
:1066D00020BD0FB6F894FA9AF99A0FBE0895019664
:1066E000272F0E945E330C945D33DC01CB01FC014B
:1066F000F999FECF06C0F2BDE1BDF89A319600B41B
:0E6700000D9241505040B8F70895F894FFCF25
:10670E00A4D0A443000000417BD49243000000417A
:10671E007BD4924300000041A4D0A443000000416A
:10672E00A4D02444000000411FD5124400000041B3
:10673E001FD5124400000041A4D0244400000041A3
:10674E00A4F076430000004100005C4300000041CD
:10675E0000005C4300000041A4F0764300000041BD
:10676E0000005C440000004148F176440000004106
:10677E005C978A44000000411FD5924400000041FE
:10678E0052D0A444000000415CFFB8440000004118
:10679E000AA7CF44000000410000DC440000004185
:1067AE00A4D082430000C0417BD49243000000413C
:1067BE00A4D0A4430000C041A4D0824300000041F5
:1067CE00A4D0A44300008041A4D0824300008041A5
:1067DE00A4D0A443000080411FD512440000804184
:1067EE00A4D024440000804100D002440000804127
:1067FE00A4D08243000080410000C44300008041C9
:10680E000AA7CF44000000410000DC440000004114
:10681E00000000000000804052D02445000040419E
:10682E0000000000000080400AA74F4500004041D4
:10683E000AA7CF44000000410000DC4400000041E4
:10684E00000000000000804052D0244500000041AE
:10685E0000000000000080405CFF38450000004151
:10686E00000000000000804052D02445000000418E
:10687E000AA7CF44000000410000DC4400000041A4
:10688E00000000000000804052D0244500008041EE
:10689E00A4F0F6430000C0417BD4924300000041B7
:1068AE0048F176440000804100005C440000004244
:1068BE005CFF434400008041A4F0F6430000C04159
:1068CE001FD51244000000415CFF4344000080418C
:1068DE005CFF384400000042A4D0A4430000804175
:1068EE00A4D0A44300008041719DAE4300008041BE
:1068FE000000C443000080410000C44300008041FA
:10690E00719DAE4300008041A4D0A443000080419D
:10691E007BD4924300008041A4D08243000080418A
:10692E00A4D08243000080417BD49243000080417A
:10693E00A4D0A44300008041A4D0A4430000C041D1
:10694E007BD49243000000417BD49243000000426E
:10695E00640007000CFF0000003F646715F515D2B8
:10696E00159E156A1501013A052808140A321E00F3
:10697E0002040507090B0C0E1011131517181A1C1B
:10698E001D1F2123242628292B2D2F303234353755
:10699E00393B1F0F03764F5F6F7F49694379392962
:1069AE001909595363333149803F5D8B803FF8BFDE
:1069BE00803FCAE1803F73ED803FCAE1803FF8BF60
:1069CE00803F5D8B803F3149803F0000803FF16DFD
:1069DE007F3F75EA7E3F4C827E3F833F7E3F842819
:1069EE007E3F833F7E3F4C827E3F75EA7E3FF16D58
:1069FE007F3F0000803F3F4D3639C7087A08440874
:106A0E000B089E07B707D007E90701020304050626
:046A1E00070809005C
:00000001FF
